:100000008DC0A7C0C0C0A5C0A4C0A3C0A2C0A1C0CD
:10001000A0C09FC09EC09DC09CC09BC09AC004034E
:100020000904580368006100660074006D006100F7
:100030006E006E00230073006F006600740077008E
:1000400061007200650020002800770077007700CB
:100050002E00740075002D006300680065006D00BF
:100060006E00690074007A002E00640065002F00A5
:100070007E0079006700750029000E0357005300C9
:1000800032003800310032003E03680065006E0027
:10009000720069006B002E00680061006600740049
:1000A0006D0061006E006E00400067006D00610031
:1000B00069006C002E0063006F006D003A00300094
:1000C0003000300031001201100100000008C0169D
:1000D000D927000101020301090222000101008069
:1000E00032090400000103000000092101010001A0
:1000F0002222000705810308000A05010909A10160
:10010000050875089504150026FF001948294B912C
:1001100002751895400501093AB102C011241FBEAD
:10012000CFE5D2E0DEBFCDBF10E0A0E6B0E0E6E470
:10013000F9E002C005900D92A436B107D9F711E09D
:10014000A4E6B0E001C01D92AF35B107E1F79BD145
:10015000F8C356CFA82FB92F80E090E041E050EAD5
:1001600060956F5F58F42D9138EF822797958795AA
:1001700010F0842795273F5FC8F3F3CF0895EADF97
:100180008D939D930895CF93CFB7CF93C395B49B91
:10019000E9F7B49B17C0B49B15C0B49B13C0B49BC4
:1001A00011C0B49B0FC0B49B0DC0C0914201C39558
:1001B000C0934201C2B7D3BBD2B3C2BBCD1BC1BB3C
:1001C000D3B3D2C00F92DF93C0914101DD27C75B4B
:1001D000DE4F012EB49B03C0DF910F90DACF2F9337
:1001E0000F931F934F932FEF4F6F06B304FB20F92C
:1001F0005F933F9350E03BE065C016B30126502962
:1002000054FDC89556B3012704FB25F92F7306B397
:10021000B1F05027102714FB26F906B22230F0F077
:1002200000C016B3012704FB27F90126502906B2A6
:100230002430E8F54F77206816B30000F6CF50273A
:100240004F7D206206B2102F000000C006B30026CA
:100250005029102714FB26F906B2E2CF4F7B06B3D4
:10026000206400C0DACF01265029187106B269F166
:100270004E7F2160012F16B328C0002650294D7FE4
:1002800006B22260102F29C0012650294B7F06B2EA
:100290002460012F2DC016B301265029477F286006
:1002A000000006B22EC04F7E06B3206130C0422748
:1002B00006B3499300265029102706B24FEF14FBCE
:1002C00020F9297F16B379F2187159F101265029C6
:1002D00006B2012704FB21F9237F06B371F2002641
:1002E00050293150D0F006B2102714FB22F9277E96
:1002F00016B351F201265029012704FB06B223F957
:100300002F7C49F2000006B3102714FB24F90026C5
:10031000502906B22F7939F270CF10E21ABF0027A8
:1003200019C03B503195C31BD04010E21ABF088161
:10033000033C01F10B34F1F020913F011981110FC1
:100340001213EDCF4A81441F093649F10D3211F0E5
:10035000013E29F7009347013F915F914F911F9113
:100360000F912F91DF910F90C0E2CABFCF91CFBF05
:10037000CF91189500914701002371F31091450129
:10038000112379F534307AF130934501009340011F
:10039000109141013BE0311B3093410124C0009199
:1003A00045010130F4F40AE54F7049F430916100E1
:1003B00034FD1AC000936100C9E2D1E019C0309148
:1003C000620034FD11C000936200C4E3D1E010C0AC
:1003D000052710E000C021C0052710E0C89508BB24
:1003E00014C03AE501C032ED032EC0E0D0E032E0A7
:1003F00017B31861C49A08B317BB58E120E84FEF50
:1004000020FF052708BB279517951C3F28F70000FC
:100410004552B0F720FF0527279508BB17951C3FCD
:10042000B8F629913A9561F7077E10914601110FB0
:1004300008BBC250D04011F010933F0110E21ABF28
:10044000006117B3177E402F477E54E05A95F1F7AD
:1004500008BB17BB48BB80CFE5E6F0E0819198E090
:10046000C09A880F9A95000008F0C09800F4000028
:10047000C09821F0000000C000C0F2CF81E0E5325A
:10048000F80761F7089584B714BE479A98E191BDC3
:1004900011BC90E195BB90E29ABF83FF09C086B37F
:1004A000887131F09BBF80E385BF78948895F8947C
:1004B00080E285BF8BE080BD82E083BF8BB7806226
:1004C0008BBF8BE48093340188E081BD86E288BBDA
:1004D000B89A85E690E060E070E040EC50E021D210
:1004E000E5E6F0E0819198E0C09A880F9A950000C7
:1004F00008F0C09800F40000C09821F0000000C08F
:1005000000C0F2CF81E0E532F80761F77894DD248E
:10051000EE24EA9445E6A42E40E0B42E32E3832E86
:1005200031E0932ECAEED0E02AE7622E20E0722E50
:1005300092E2492E90E0592E8EE1282E80E0382E4E
:1005400001C0DC2C86B3887109F08895C090420107
:10055000A8959091450119160CF026C18091410192
:10056000ECE0F0E0E81BF109E75BFE4F092F0350D8
:10057000809140018D3209F0BDC09AE590936100F1
:10058000083009F007C19081892F807609F085C075
:10059000109232018181882349F4109233019092A4
:1005A00044018092430120E892E099C0853021F413
:1005B00082818093460191C0863009F050C08381CA
:1005C000813049F486EC90E090934401809343019C
:1005D00020EC92E184C0823019F488ED90E038C0BC
:1005E000833041F58281882339F43092440120928E
:1005F000430120EC94E073C0813039F450924401FF
:100600004092430120EC98E56AC0823039F4709240
:1006100044016092430120EC9EE061C0833009F008
:100620005AC088E890E0909344018093430120EC05
:100630009EE355C0813239F4D0934401C093430105
:1006400020EC99E04CC0823209F045C08AEF90E07E
:10065000909344018093430120EC92E240C08830A3
:1006600039F488E491E090934401809343010CC0F5
:10067000893021F48281809348012FC08A3039F477
:10068000909244018092430120E891E028C08B3091
:1006900021F59BE49093340120C0892F807680322D
:1006A000E1F48181813039F4B0924401A092430198
:1006B00020E890EC14C0893081F483818093250177
:1006C000B0922701A092260166816093280197FDD0
:1006D0000AC06FEF08C020EC01C020E890E08781DD
:1006E000882319F05AC020E059C06681691708F4C0
:1006F00055C053C08091640087FD4CC08091250196
:100700008230C9F41092250180912801843008F4C8
:100710003FC00430E8F183818034D0F590E063E09D
:1007200070E0E4D0DC01AB59BF4F83E001900D9243
:100730008150E1F72BC0833009F0D2C080912801AD
:10074000882309F4CDC0002309F4CAC0F02E801715
:1007500008F4F82E0F2D10E08091260190912701CA
:10076000BF014F2D50E0D4D08091260190912701F8
:10077000800F911F9093270180932601809128017B
:100780008F1980932801882309F0ADC0E0922501DC
:1007900020E001C020E860E001C0692F20936400E0
:1007A00060936000109245018091610084FF48C011
:1007B000809160008F3F09F443C0082F893008F012
:1007C00008E0801B809360008091640080FD02C07F
:1007D0001BE401C013EC8F5F809364002091430100
:1007E0003091440186FD05C0D901902FEAE2F1E085
:1007F00011C0AAE2B1E080E090E006C0F901E80F84
:10080000F91FE491ED9301960817C1F705C08D918A
:10081000819391509923D9F7F901E00FF11DF093DD
:100820004401E09343018AE291E0602FA8DC0830A4
:1008300011F0E0926000109329010C5F00936100B9
:100840009AE086B3887131F49150D9F7109246013D
:1008500010923F01CD1409F475CE91B39E50993F8B
:100860001CF481B78F5F81BF98301CF081B7815035
:1008700081BF809125018F3FD9F4F894E5E6F0E03F
:10088000819198E0C09A880F9A95000008F0C0986E
:1008900000F40000C09821F0000000C000C0F2CFBA
:1008A00081E0E532F80761F778941092250149CE8E
:1008B000E19947CEEEB3EF5FE03C08F0E0E0F0E016
:1008C000FFBBEEBBE09A8DB3EB59FF4FE0818E1773
:1008D00009F437CEEDBBF894E29AE19A789431CEE0
:1008E0009EE19093610020E06FEF58CF55270024E0
:1008F00080FF02C0060E571F660F771F6115710536
:1009000021F096958795009799F7952F802D08955A
:10091000FB01DC0102C001900D9241505040D8F71C
:100920000895DC01CB01FC01E199FECF06C0FFBBBD
:10093000EEBBE09A31960DB20D9241505040B8F79F
:060940000895F894FFCFBA
:04094600FF5A5A00FA
:00000001FF
